:100000000C946D010C94A5010C94A5010C94A50110
:100010000C94A5010C94A5010C94A5010C94A501C8
:100020000C94A5010C94A5010C944C1E0C941E1F5D
:100030000C945E190C94A5010C94A5010C94A501D7
:100040000C94A5010C94A5010C94A5010C94A50198
:100050000C94A5010C94E6190C94A5010C94A5012F
:100060000C94A5010C94A5010C94A5010C94A50178
:100070000C94A5010C94A5010C94A5010C94A50168
:100080000C94A5010C94A5010C94A5010C94A50158
:100090000C94A5010C94A5010C94A5010C94A50148
:1000A0000C94A5010C94A5010C94A5016C046C049E
:1000B0009804980400052B062B062B061E05B70591
:1000C000C805C8058B1FB21FAA20B21FAA20FE1F99
:1000D0002120AA20782087200400C35C06001B0092
:1000E0001C001D00000101010101010101010202CA
:1000F00002020202020202030303030303030304D6
:1001000004040404040405050505050606060606A0
:10011000070707070708080808090909090A0A0A5A
:100120000B0B0B0C0C0C0D0D0D0E0E0E0F0F0F10FC
:100130001011111112121313141415151616171786
:10014000181819191A1A1B1B1C1D1D1E1E1F2020F2
:10015000212222232424252626272829292A2B2C3C
:100160002D2D2E2F30313232333435363738393A5F
:100170003B3C3D3E3F404142434445464748494A57
:100180004C4D4E4F50515354555658595A5B5D5E25
:100190005F616264656668696B6C6D6F70727375C0
:1001A00077787A7B7D7E8082838587888A8C8E8F24
:1001B00091939596989A9C9EA0A2A3A5A7A9ABAD52
:1001C000AFB1B3B5B7BABCBEC0C2C4C6C9CBCDCF40
:1001D000D1D4D6D8DBDDDFE2E4E7E9EBEEF0F3F5EE
:1001E000F8FAFDFF180345006C006C006900700010
:1001F00073006500520065007600310000001603B0
:1002000041006200730074007200610063007400BA
:100210004B00420000000403090409023B000201F4
:1002200000A0FA09040000010301010009211101E5
:1002300000012240000705810308000109040100B4
:10024000010300000009211101000122320007050D
:1002500082032000011201000200000008EDFE01EF
:100260000001000102000105010980A101850319B7
:10027000012AB700150126B700950175108100C04D
:10028000050C0901A101850419012AA00215012606
:10029000A002950175108100C005010906A10105A4
:1002A0000719E029E71500250195087501810295D8
:1002B00001750881010507190029FF150026FF00B7
:1002C0009506750881000508190129059505750130
:1002D0009102950175039101C00011241FBECFEF5B
:1002E000DAE0DEBFCDBF04B603FE18C08091510234
:1002F00090915202A0915302B09154028730904BDA
:10030000A740B04B59F41092510210925202109231
:10031000530210925402E0E0F8E3099511E0A0E0E6
:10032000B1E0E6ECF2E402C005900D92A639B10707
:10033000D9F722E0A6E9B1E001C01D92A135B207CC
:10034000E1F70E94CE110C9461210C940000811100
:1003500006C0662311F082E113C083E111C0813031
:1003600041F4662319F00E94A3130CC00E94B3133A
:1003700009C0823039F4662311F080E101C085E1C3
:100380000E941A0481E0089581E0089581E00895B3
:100390000C94C60108950C94CA011F93CF93DF9368
:1003A00000D000D01F92CDB7DEB749835A836B834C
:1003B0003091990189819A81311114C0662359F0D5
:1003C000222349F00E946408182F682F89819A819E
:1003D0000E940D0803C00E943808182F69817A8195
:1003E000812F04C00E94640869817A810F900F9068
:1003F0000F900F900F90DF91CF911F910C94890F68
:10040000FC01262F408151816281738184810C948B
:10041000CD0181E00895CF93DF93EC0160E00E946D
:100420000002BE01DF91CF910C94CB010C94B81067
:100430000C94B41008950E94B7060E941A022FEF80
:1004400084E39CE0215080409040E1F700C0000030
:100450000C940C1A0F931F93CF93DF938C0161E0E0
:100460000E940002EC01B8010E94C801882309F42F
:1004700044C0B801CE010E9436188823F1F1B801BA
:10048000CE010E9427158823C1F1B801CE010E9438
:100490009217882391F1B801CE010E948514882318
:1004A00061F1F8018281882309F1CB358DE5D80708
:1004B000C1F050F4C115FCE5DF0781F0CF3DDC450C
:1004C000A9F40E94950D19C0CC35EDE5DE0761F069
:1004D000CD35DD4559F40E94DE0C08C00E941B0298
:1004E0000CC00E94E70C02C00E94EA0CC801DF9118
:1004F000CF911F910F910C94C40180E0DF91CF91B7
:100500001F910F9108950E943F190E94A0020C9420
:100510002B130E94A3020E9477140C94451908958E
:100520000C948F0281E008950C9492020895CF9369
:10053000C82F0E9490028C2F0E949402CF910895A0
:1005400080E00C9497020E9492180C9497020E94EB
:10055000921890919801891721F0809398010C943A
:1005600097020895CF93DF93CDB7DEB72B970FB6E1
:10057000F894DEBF0FBECDBF4F83588769877A8757
:100580008B8761110E942A0C9E012F5F3F4F86E0EE
:10059000F90111928A95E9F785E0FE013796D901B4
:1005A00001900D928A95E1F789819A814C815D8154
:1005B000452B31F09F3F31F491E08F3F19F403C098
:1005C00091E001C090E090FF09C049815A816B81A0
:1005D0007C818D819E810E944B0B05C0C9010E94C8
:1005E00009028111F2CF2B960FB6F894DEBF0FBE31
:1005F000CDBFDF91CF910895FC01808191810E9450
:10060000A6080895CF93882309F49CC0C82F823888
:10061000C1F40E94921881FD95C069E380910201A6
:10062000909103010E9417190E944C0C2FEF81EE4C
:1006300094E0215080409040E1F700C0000069E361
:1006400019C0833801F50E94921880FD7BC063E5D4
:1006500080910201909103010E9417190E944C0C95
:100660002FEF81EE94E0215080409040E1F700C0F0
:10067000000063E580910201909103010E94191925
:10068000CF910C944C0C8438C1F40E94921882FDD6
:1006900059C067E480910201909103010E941719EB
:1006A0000E944C0C2FEF81EE94E02150804090404E
:1006B000E1F700C0000067E4DDCF8CEF8C0F813ADA
:1006C000D0F46C2F80910201909103010E94E118F7
:1006D000882349F06C2F80910201909103010E94C0
:1006E00019190E944C0C6C2F80910201909103010A
:1006F0000E941719C5CF80E28C0F883048F4C7706C
:1007000081E001C0880FCA95EAF70E940D0CB8CFAE
:10071000EBE5EC0FE33040F4F0E0EC5BFE4F808162
:1007200090E0CF910C94A918C85AC73158F4EC2F17
:10073000F0E0EE0FFF1FEA5EFE4F80819181CF91C6
:100740000C94BF18CF910895882309F45BC0682FDB
:10075000823879F40E94921881FF54C069E3809135
:100760000201909103010E9417190E944C0C69E349
:1007700010C08338B1F40E94921880FF43C063E533
:1007800080910201909103010E9417190E944C0C64
:1007900063E580910201909103010E9419190C9464
:1007A0004C0C843879F40E94921882FF2BC067E4C5
:1007B00080910201909103010E9417190E944C0C34
:1007C00067E4E7CF8CEF860F813A18F380E2860F5B
:1007D000883048F4677081E001C0880F6A95EAF7B5
:1007E0000E94130CDCCF8BE5860F833020F480E071
:1007F00090E00C94A918685A673120F480E090E0EA
:100800000C94BF1808951F93CF93DF93182FEB011B
:100810000E940203209741F08FE99FE00197F1F7D2
:1008200000C000002197F6CF812FDF91CF911F915B
:100830000C94A403893319F060E070E002C060E515
:1008400070E00C940304882321F00E940D0C0C949A
:100850004C0C0895882321F00E94130C0C944C0C2E
:100860000895CF92DF92EF92FF920F931F93CF9351
:10087000DF937C01D62FC72FFC01128105810295E1
:100880000F700E94030C8823B9F01123A9F08C2F5C
:10089000807F803421F080E28D0F883068F0809175
:1008A0002D0282FD09C082E00E94AC0C0E94030C64
:1008B00091E0D82ED92601C0D12CCC2EC2948FE045
:1008C000C8228C2D90E08C30910508F0C4C1FC0149
:1008D000EA5AFF4F0C9406218C2F807FCF7088231B
:1008E00011F0C295C07F112399F0CC2309F49FC168
:1008F00080E28D0F883010F0D11104C08C2F0E943F
:100900000D0C03C08C2F0E941D0C0E944C0C8FC13B
:100910008D2F0E94A403CC2309F49DC180E28D0F8A
:10092000883038F1DD2329F18C2F0E94230C24C05C
:100930008C2F807FCF70803211F0C295C07FDD2375
:1009400019F0D130A1F13DC080912D0282FF17C076
:10095000112349F0CC2329F08C2F0E940D0C0E940A
:100960004C0C80E065C180E00E94A403CC2309F414
:1009700072C18C2F0E94130C0E944C0C6CC111236D
:1009800071F0002341F0013031F40E942D0C8C2BCA
:100990000E94350C60C10E942D0C8C2B1DC00023C1
:1009A00019F0013009F457C10E94420C25C01123EF
:1009B00021F0063008F04FC10EC0053008F04BC1E1
:1009C0001BC0112361F0002331F0F701858180FF06
:1009D0002EC18F7085838C2F0E9423043CC100237D
:1009E00059F0D93309F034C1FFEF07EE13E0F150AD
:1009F00000401040E1F72AC18C2F0E942A042BC12D
:100A00008C2F86958695837019F0813061F023C113
:100A1000112321F08D2F9C2F937002C080E090E075
:100A20000E94A91820C1112321F08D2F9C2F9370B3
:100A300002C080E090E00E94BF1815C18C2F837027
:100A400009F047C011110BC12D2F22952695277053
:100A5000220F220F6D2F6F70862F90E0A0E0B0E084
:100A6000022E04C0880F991FAA1FBB1F0A94D2F739
:100A7000D4FF10C04FE050E060E070E004C0440FCD
:100A8000551F661F771F2A95D2F7409550956095A0
:100A9000709503C040E050E0BA01C695C695C3709A
:100AA0008A019B01082B192B2A2B3B2BC901B8016A
:100AB000C23049F058F4C13019F00E942307CFC06A
:100AC0000E941107CCC00E943507C9C00E940F07C1
:100AD000C6C0112319F08C2F817001C08695882320
:100AE00009F4BDC02D2F229526952770220F220FC5
:100AF0006D2F6F70862F90E0A0E0B0E0022E04C052
:100B0000880F991FAA1FBB1F0A94D2F7D4FF10C0E9
:100B10004FE050E060E070E004C0440F551F661FD6
:100B2000771F2A95D2F7409550956095709503C030
:100B300040E050E0BA01C695C695C3708A019B019A
:100B4000082B192B2A2B3B2BC901B801C23049F0C5
:100B500058F4C13019F00E94E80781C00E94D607FE
:100B60007EC00E94FA077BC00E94490778C0CF7000
:100B7000112339F08C2F0E946F078D2F0E942304C0
:100B80006EC08D2F0E942A048C2F0E94900767C090
:100B9000D23F21F128F4D03F41F0D13FC1F043C012
:100BA000D33F19F1D43F79F03EC0112341F0053015
:100BB00008F051C08C2F8F710E94B5074CC00630D1
:100BC00008F049C0F7CF80912D0282FF18C0112391
:100BD00039F08C2F8F710E946F073DC01123C9F32C
:100BE0008C2F8F710E94900736C0112329F08C2F13
:100BF0008F710E945A072FC00E9455072CC01123E5
:100C000049F0CF718C2F0E946F0763E08C2F0E94F8
:100C1000910C21C081E00E94AC0C0230E0F082E037
:100C20000E94AC0C18C0112331F0002391F28D2FDB
:100C30000E94020310C0002399F2D93349F41FEF38
:100C400027EE33E0115020403040E1F700C00000B3
:100C50008D2F0E94A40388EF8C0D843020F40E9415
:100C600092180E949702DD20C9F00E94FF0B80FDC0
:100C700015C0F70112820E94F90B0E946F07C7018D
:100C80000E946F060E94F90BDF91CF911F910F9187
:100C9000FF90EF90DF90CF900C949007DF91CF9171
:100CA0001F910F91FF90EF90DF90CF9008950F93D9
:100CB0001F93CF93DF93EC01688179818A810E9431
:100CC000B1088C010E940C080E94FD06B801CE01FB
:100CD0000E943104DF91CF911F910F910895CF931E
:100CE000DF93EC01988189812B813C81232B31F0AA
:100CF0008F3F31F481E09F3F19F403C081E001C0D0
:100D000080E080FD1DC0CE010E942A02811110C02A
:100D10000E94030C8823A1F08A81882389F08091A6
:100D20002D0282FD0DC082E0DF91CF910C94AC0CBE
:100D3000CE010E945706CE01DF91CF910C940B0299
:100D4000DF91CF91089580E090E00E94A91880E0A3
:100D500090E00E94BF180E942A0C0C944C0C8091C9
:100D60000201909103010E941B190C94A3060E949A
:100D70001A0C0C94AF0692959F70963079F010F48F
:100D8000925001C09A50923068F4803F69F018F494
:100D9000883E40F409C0843F29F406C0883E20F014
:100DA000813F11F080E0089581E00895FC01808189
:100DB00091810E94A6080E94BB060895CF93DF93FD
:100DC00000D000D01F92CDB7DEB70F900F900F90DC
:100DD0000F900F90DF91CF910895CF93DF9300D0C4
:100DE00000D000D0CDB7DEB726960FB6F894DEBFA0
:100DF0000FBECDBFDF91CF910895089508950C9453
:100E0000FE060C94FF060E9401076093A3017093F5
:100E1000A4018093A5019093A6010C94A3060C94C1
:100E200003070F931F930091A3011091A401209138
:100E3000A5013091A601602B712B822B932B1F9162
:100E40000F910C9403070F931F930091A30110912E
:100E5000A4012091A5013091A60160237123822372
:100E600093231F910F910C9403070F931F930091ED
:100E7000A3011091A4012091A5013091A601602742
:100E80007127822793271F910F910C9403070C94CD
:100E9000FE060E94470760939F017093A001809314
:100EA000A1019093A2010C94A30660E070E0CB0135
:100EB0000C9449070F931F9341E050E060E070E00D
:100EC0008A019B0104C0000F111F221F331F8A9546
:100ED000D2F7C901B8011F910F910C9449070F93E4
:100EE0001F9341E050E060E070E004C0440F551FE4
:100EF000661F771F8A95D2F780919F019091A0017C
:100F0000A091A101B091A2018A019B01082B192B8C
:100F10002A2B3B2BC901B8011F910F910C94490753
:100F20000F931F9341E050E060E070E004C0440F75
:100F3000551F661F771F8A95D2F74095509560958B
:100F4000709580919F019091A001A091A101B09115
:100F5000A2018A019B01082319232A233B23C901EB
:100F6000B8011F910F910C9449070F931F9341E013
:100F700050E060E070E004C0440F551F661F771F0B
:100F80008A95D2F780919F019091A001A091A10133
:100F9000B091A2018A019B01082719272A273B2724
:100FA000C901B8011F910F910C9449070F931F932A
:100FB00000919F011091A0012091A1013091A20107
:100FC000602B712B822B932B1F910F910C9449074F
:100FD0000F931F9300919F011091A0012091A101F7
:100FE0003091A20160237123822393231F910F91DB
:100FF0000C9449070F931F9300919F011091A0013A
:101000002091A1013091A2016027712782279327A7
:101010001F910F910C9449070895292F220F920FC9
:10102000890FE82FE695E695E695877051E001C0B7
:10103000550F8A95EAF785E0E89FF0011124E656FE
:10104000FE4F20E030E070E04081CB01022E02C074
:10105000969587950A94E2F7817081958427852378
:10106000842781932F5F3F4F2530310569F708951D
:10107000292F220F920F890F682F66956695669526
:10108000982F977085E0689FB001112440E050E0F0
:1010900080E0FB01E40FF51FE656FE4F208130E0B3
:1010A000092E02C0369527950A94E2F7217033275E
:1010B000042E01C0220F0A94EAF7822B4F5F5F4F84
:1010C0004530510531F70895BF92CF92DF92EF92EC
:1010D000FF920F931F93CF93DF938C01C0909F01DA
:1010E000D090A001E090A101F090A2018091A30115
:1010F0009091A401A091A501B091A601C82AD92A76
:10110000EA2AFB2ACFE1D0E0D701C6010C2E04C0A9
:10111000B695A795979587950A94D2F780FD04C058
:10112000219790F7B12C07C0BC2EB8018C2F0E94DC
:101130009F0F0197A9F38B2DDF91CF911F910F91F5
:10114000FF90EF90DF90CF90BF900895CF93DF9303
:10115000EC010E946408BE010E949F0FDF91CF91B5
:1011600008951F93CF93DF93EB01909199019923F9
:1011700021F0CB010E94A60813C0882349F0CB01BF
:101180000E946408182F682FCE010E940D0804C029
:10119000CB010E943808182FBE01812F0E949F0F9B
:1011A000DF91CF911F9108951F93CF93DF93C0914B
:1011B000A70116E08091A801C81799F0D0E01C9F04
:1011C000F0011D9FF00D1124E755FE4F4081518124
:1011D00062817381848195810E94ED062196C7709A
:1011E000E9CFDF91CF911F9108954091D90150919E
:1011F000DA016091DB017091DC018091DD01909159
:10120000DE010C94ED06EF92FF920F931F93CF93A4
:10121000DF938091DE0182958F7009F065C0809127
:10122000DB01882309F460C08091A701F090A80138
:101230001091D9010091DA016091DC017091DD011A
:1012400091E01F3F09F090E0C0910001D0910101B1
:10125000292F96E0E92E8F1509F446C06115710516
:1012600021F00F3F21F030E003C031E001C0322F08
:1012700090E030FD36C0E89EF001E99EF00D1124AB
:10128000DF01A755BE4F11963C911197301329C02D
:101290003C91311326C012963C911297311121C016
:1012A00013964D915C911497461B570B4C175D0795
:1012B000C0F48091DE018F7080618093DE01E25581
:1012C000FE4F80818F708061808389ED91E00E9464
:1012D0006F06DF91CF911F910F91FF90EF900C94CB
:1012E000D40801968770B7CFDF91CF911F910F91EE
:1012F000FF90EF9008959F92AF92BF92CF92DF92AE
:10130000EF92FF920F931F93CF93DF93CDB7DEB78A
:1013100061970FB6F894DEBF0FBECDBF8C0185E09C
:10132000F801DE011D9601900D928A95E1F7D80132
:101330001296EC909091D901E091DA012091DC01B4
:101340003091DD012115310531F0EF3F31F481E0BD
:101350009F3F19F403C081E001C080E0B82FB17055
:101360009B2E80FD47C1D8014C9111965C9111973D
:101370001396AD90BC90149789EDC82E81E0D82EBD
:10138000F090DB01B501621B730B209100013091DD
:101390000101FF2009F4D9C08091DE0162177307B3
:1013A00008F095C0282F207F09F052C05E1313C0AB
:1013B000491311C0FE2CE1100EC08F708061809324
:1013C000DE010E94F508C6010E946F068091DE01D1
:1013D000F80185834DC1AB2831F05F3F31F481E0E6
:1013E0004F3F19F403C081E001C080E080FD03C0DD
:1013F00081E08E2502C080E090E0F82FF170FF2E92
:1014000080FF1CC08091A7012091A80136E08217BF
:1014100009F40BC190E0389FF001399FF00D1124C1
:10142000E755FE4F6181561306C06081461303C025
:101430006281E61203C001968770E9CFFE2CEE2090
:1014400009F416C18091DE0181608093DE0154C0F1
:101450005E1306C0491304C0E11002C0F80199C030
:10146000C8010E94D606882361F1EE2051F1209137
:10147000DE01822F82958F7090E0029774F0809148
:10148000D9019091DA0198878F831986BB86AA8645
:101490002C87CE0107960E946F0686E0F801A9ED21
:1014A000B1E001900D928A95E1F70E9403090E9434
:1014B000F5080AC05E1711F1C8010E94D606811115
:1014C0002CC0C8010E946F06FF24F394D1C0282FBE
:1014D000207F81F77A2DB98AA88A6E2D89890E948A
:1014E000DE0689ED91E00E946F0686E0D6011D922E
:1014F0008A95E9F70E94F508F12CBAC04913DCCFB0
:10150000E110DACFF8018583C8010E946F0686E0FA
:10151000D6011D928A95E9F7ABC0EE2091F2209199
:10152000DE01822F82958F7090E002970CF4B5CF88
:101530008091D9019091DA019A8389831B82BD82BF
:10154000AC822E83CE010196A6CF6217730708F0F6
:1015500044C0FE2CEE2009F4B4CF5E1330C0491312
:101560002EC02091DE0120FD21C0822F82958F7038
:10157000482F50E041155105C9F0F80125834F303F
:10158000510541F08F5F982F9295907F822F8F7039
:10159000892B8583C8010E946F0686E0F801A9EDBA
:1015A000B1E001900D928A95E1F73CC086E0F80128
:1015B000A9EDB1E001900D928A95E1F759C0C801FB
:1015C0000E94D606811169CF8091DE0181608093EF
:1015D000DE01C8010E946F064BC07A2DB98AA88A25
:1015E0006E2D89890E94DE0686E0D6011D928A95BD
:1015F000E9F718C0EE2009F464CFC8010E94D606AE
:10160000F82E882309F45DCF86E0F801A9EDB1E05A
:1016100001900D928A95E1F789ED91E00E94FC021C
:101620000E9403090E94F50823C04D875E878D85BF
:101630009E850E94A608292F22952F70223028F41B
:101640009F7039F0811105C00BC0243028F49F70C1
:1016500049F4805E883020F0C8010E946F069F2CFC
:10166000F92C06C0D80115969C91907F91F7F8CF80
:101670008F2D61960FB6F894DEBF0FBECDBFDF9100
:10168000CF911F910F91FF90EF90DF90CF90BF907F
:10169000AF909F9008951F93CF93DF93CDB7DEB7A0
:1016A0002C970FB6F894DEBF0FBECDBF4F8358877F
:1016B00069877A878B879C87CE0107960E947B0972
:1016C0008823D1F09F8188852A853B85232B31F0A3
:1016D0008F3F31F481E09F3F19F403C081E001C0E6
:1016E00080E080FD47C04F81588569857A858B856C
:1016F0009C850E94ED063EC086E0FE013796DE0125
:10170000119601900D928A95E1F7FF81E8856A852F
:101710007B856115710531F0EF3F31F481E0FF3FCA
:1017200019F403C081E001C080E080FD23C0209156
:10173000A80130E0C9010196877099274091A7015F
:1017400050E084179507F1F1F983EA837D836C8378
:1017500096E0929FD001939FB00D1124A755BE4FE4
:10176000FE01319601900D929A95E1F78093A801C0
:101770000E94D40816E08091A7019091A8018917D2
:1017800071F1189FC001112487559E4F0E947B095B
:10179000882329F1E091A7011E9FF0011124E7554C
:1017A000FE4F4081518162817381848195810E94C5
:1017B000ED068091A70190E00196877099278093AC
:1017C000A701D9CF0E94B7061092A8011092A701D5
:1017D000E9EDF1E086E0DF011D928A95E9F72C96AC
:1017E0000FB6F894DEBF0FBECDBFDF91CF911F9132
:1017F00008958091E7018595859585950895809157
:10180000E701877008959091E701977081E009F4EE
:1018100080E008958091F20108959091F201892B62
:101820008093F201089580959091F201892380932D
:10183000F20108951092F20108959091F101892B1F
:101840008093F101089580959091F101892380930F
:10185000F10108951092F10108958091E801089531
:1018600008950C94300C0C94310C90912D0292FD43
:1018700008C09091E801981721F08093E8010C943A
:10188000330C08958091E801882329F01092E80133
:1018900080E00C94330C0895CF93DF93E091020124
:1018A000F09103018091F2018083E0910201F091B7
:1018B000030190818091F101892B80838091E8015F
:1018C000882381F0E0910201F09103019081892B3E
:1018D000808380910201909103010E94D5188111AB
:1018E0000E94420CC0910201D091030148E050E0F7
:1018F0006FED71E0CE010E940C21892B69F088E028
:10190000FE01AFEDB1E001900D928A95E1F7CE01B5
:10191000DF91CF910C949E18DF91CF9108950C9494
:10192000300C90912D0292FD10C098E0899F90019B
:101930001124262B2093E7010E946F078091E70175
:101940008595859585950C948F0C0C946F07109256
:10195000E70180E00C948F0C2091E70180958223B1
:101960008093E701982F977099F430E0482F082E64
:10197000000C550B2417350759F090912D0292FD5C
:1019800007C08595859585950E9490070C94A70CB6
:10199000089590912D0292FB222720F9281769F0D3
:1019A00080FB92F990932D0280912C0290912D0250
:1019B0000E94110D82E00C94AC0C089580912D02D0
:1019C00082FB882780F991E089270C94C90C81E07B
:1019D0000C94C90C80E00C94C90C80E090E00E944B
:1019E000272121E0893E9E4F09F020E0822F0895B3
:1019F00082E090E00C94192183E090E00C9419218E
:101A0000CF9384E090E00E941921C82F82E290E0F9
:101A10000E9419212C2F30E0A901582BCA01CF9127
:101A20000895CF93C92F682F84E090E00E942D2164
:101A30006C2F82E290E0CF910C942D21AB01BC0180
:101A40008FE090E00C943F21AB01BC0183E190E07A
:101A50000C943F2160E070E0CB010C94240D60E019
:101A600070E0CB010E941E0D0C942A0D69EE7EEFF2
:101A700080E090E00E944B2160E082E090E00E94D4
:101A80002D2160E083E090E00E942D211092A301BF
:101A90001092A4011092A5011092A60160E084E0CA
:101AA00090E00E942D2160E082E290E00E942D21D2
:101AB00060E085E090E00E942D2160E086E090E00B
:101AC0000E942D216FEF87E090E00E942D2140E0E1
:101AD00050E0BA0188E090E00E943F2160E08DE094
:101AE00090E00E942D2140E050E0BA0188E190E0B2
:101AF0000E943F2160E087E190E00E942D2140E0BC
:101B000050E0BA018CE190E00E943F2160E070E07B
:101B100080E290E00E944B2140E050E0BA0188E171
:101B200090E00E943F210C942F0D0C94360D682FED
:101B30008EE090E00C942D210E94CB196093FD0162
:101B40007093FE018093FF01909300026093F9016E
:101B50007093FA018093FB019093FC0108950E9419
:101B6000CB196093FD017093FE018093FF01909368
:101B700000026093F5017093F6018093F701909352
:101B8000F801089585B7806885BF85B7806885BFEF
:101B9000089581E008950C94C90D08950C94CD0D1D
:101BA0000C94CD0D0C94D00D0C94CD0D0C94D40D43
:101BB0000C94CD0D0E94C20D8BE790E10E94881815
:101BC0000E94D80D0C94D60D0E94CE0D0C94CD0D14
:101BD0000E947E100C9496020E94B6190E94441135
:101BE0000E94E80D0E943E140E9478160C94D20DBB
:101BF0008F929F92AF92BF92CF92DF92EF92FF921D
:101C00000F931F93CF93DF93CDB7DEB72A970FB60D
:101C1000F894DEBF0FBECDBF0E945311982E8111E4
:101C20000E949C0D83EFA82E81E0B82E00E010E00A
:101C3000802E802F0E94A210D82EF501C1905F0146
:101C4000C826B1F40F5F1F4F0230110589F78FEFDF
:101C500089838A831B820E94BF198160782F9D83AC
:101C60008C8349815A816B818D810E94B2022FC081
:101C70008091010281FD0E94A810E12CFF24F394C1
:101C80008C2D8F21F1F00E94CB0D882399F0EE82EC
:101C90008F82DF2081E009F480E088870E94BF19ED
:101CA0008160782F9A8789874E815F8168858A85D0
:101CB0000E94B202F801ED50FE4F8081F826F082BA
:101CC00006C0E394FF0CF3E0EF12DACFBBCF81E064
:101CD000911001C080E02A960FB6F894DEBF0FBEC7
:101CE000CDBFDF91CF911F910F91FF90EF90DF90CB
:101CF000CF90BF90AF909F908F9008950E94F80D65
:101D00000E94ED1681110E94AF0D0C94A702CF9393
:101D1000DF930E94A40FEC01811522E59207E8F5FC
:101D2000811531E5930708F0B6C0883E910528F586
:101D3000803E910508F0E9C0883A910570F4853A33
:101D4000910508F07AC08130910509F473C008F458
:101D5000D9C0049708F0D9C0D5C08F3B910508F0D1
:101D6000D1C0C85AD0E0CC0FDD1FC95BDE4F09904F
:101D7000D881C02DCE019464C9C0811540E5940777
:101D800008F069C0811550E4950708F060C09A9585
:101D900081159F4108F4B9C0B5C0811536E5930798
:101DA00028F5811545E5940708F092C0811554E5A2
:101DB000950708F087C0AC0143705527282F26955A
:101DC0002695C115D34508F06CC081E090E002C0B3
:101DD000880F991F4A95E2F740E2249F9001112451
:101DE000EC01C22BD32BCE019C6890C081152AE553
:101DF000920780F4811539E5930708F072C08115C8
:101E000048E5940708F47EC0D82FCC27CE01806F18
:101E1000906A7CC090568115904208F073C08D2F57
:101E20008F710E943810DD27D0628F71AE01582B60
:101E3000CA016CC081E090E069C0C55AD0E0CB58BF
:101E4000DE4F8881C82FD0E0CE0190645FC0DF7084
:101E5000CE01906A5BC074E0969587957A95E1F71C
:101E6000282F23703C2F337081E090E002C0880F50
:101E7000991F3A95E2F79C68AC01522B9A019C2F6E
:101E80009F709695969550E2959FE0011124C901A7
:101E90008C2B9D2B3BC0D82FCC27CE01816F906A15
:101EA00035C081E090E002C0880F991F4A95E2F7A3
:101EB00050E2259F90011124EC01C22BD32BCE01BF
:101EC0009A6824C0D82FCC27CE01846F906A1EC098
:101ED0000E9438108F7190E0D82FCC27CE019062ED
:101EE00015C08F700E94381094E0D695C7959A95CA
:101EF000E1F7CF70D0E0DC2FCC27D0699E01282BF2
:101F0000C90104C080E090E001C0CE01DF91CF9113
:101F10000895272F30E0F901EE0FFF1F2E0F3F1F0E
:101F2000F90196E0899FE00DF11D1124E60FF11DE6
:101F3000EE0FFF1FE852FF4F8591949108950E9484
:101F4000890F0E94870E08958238910569F1B0F4D7
:101F50008133910509F46DC048F48932910509F483
:101F600063C08A32910509F469C0089585339105EB
:101F700009F455C089339105B9F00895833E910560
:101F800069F138F4803E9105B1F0823E910509F186
:101F90000895863E9105A9F1873E9105B9F1843EE9
:101FA000910509F064C023C020912C0220FD4FC090
:101FB00021FD4DC0089580912C0280FD44C0809188
:101FC0002D0280FF44C080912C0284FD42C083EE2C
:101FD0004DC080912C0282FF38C0F5CF80912C0239
:101FE00082FD33C080912D0280FD31C0ECCF809105
:101FF0002D0281FF32C080912C0284FD2AC087EE21
:1020000035C080912C0283FF26C0F5CF80912C0231
:1020100083FD21C080912D0281FD1FC0ECCF8091F6
:102020002C0285FD1CC01DC080912C0285FD19C0AD
:1020300016C080912C0286FD16C017C080912C021C
:1020400086FD13C010C089E311C082EE0FC080EE80
:102050000DC080E00BC086EE09C084EE07C089E2A7
:1020600005C085E303C08AE201C081E390E00895E2
:1020700090912C0292FF0DC0282F2871283019F45E
:10208000877F846006C0282F2471243011F48B7F51
:10209000886093FF0DC0282F2871283119F4877E9E
:1020A000846106C0282F2471243111F48B7E88614D
:1020B00020912D0220FF0DC0382F3871383019F4CF
:1020C000877F816006C0382F3171313011F48E7FE7
:1020D000886021FF0DC0282F2871283119F4877ED0
:1020E000816106C0282F2171213111F48E7E886113
:1020F00094FD877E089580E0089508950E94ED0C78
:10210000811102C00E94950D0E94F80C809301027B
:102110000E94000D90932D0280932C020E947D104E
:102120000E94FC0C682F70E080E090E00E940F0796
:1021300060919F017091A0018091A1019091A201F5
:102140000C944707E82FF0E0E05DFD4F8081089593
:10215000089580EA8A95F1F7089500C008950C94D7
:10216000A91008950C94B1100C94B2100C94B110F5
:102170000C94B610F894E82FE295EF70F0E031A1DE
:10218000282F2F7081E090E001C0880F2A95EAF790
:10219000982F9095932391A392A1892B82A3789451
:1021A000089583E90E94BA1087E60E94BA1080EF72
:1021B0000E94BA1086E30E94BA1085E30C94BA100C
:1021C000CF92DF92EF92FF920F931F93CF93DF9303
:1021D0008C01C62FD0E0CE0185589E4F7C01FC01BA
:1021E00090819F3F09F447C0D62EF894E92FE295DD
:1021F000EF70F0E081A19F7021E030E001C0220F7C
:102200009A95EAF7822B81A382A12095282322A305
:1022100078940E94AD10E8E7F1E04BE751E031E03F
:10222000C12C21912F3F89F0A22FA295AF70B0E071
:1022300090968C9190E02F7002C0959587952A9585
:10224000E2F780FD02C0832F01C080E0C82A330F6F
:102250004E175F0731F7F70180818F3F11F00E9421
:10226000BA1061E0C11001C060E08D2D0E94AF1076
:10227000C00FD11FC882DF91CF911F910F91FF90A6
:10228000EF90DF90CF9008950E94D110109231020C
:102290001092300210922F0210922E0282E00E94C1
:1022A0008B110C9416021F93CF93DF9300D0CDB700
:1022B000DEB71A82198260E0CE0101960E94E0101A
:1022C00061E0CE0101960E94E01042E050E0BE01C4
:1022D0006F5F7F4F8EE292E00E940C2111E0009729
:1022E00009F410E0892B31F089819A8190932F02B3
:1022F00080932E02212F42E060E372E08EE292E0B2
:102300000E948C110E941802812F0F900F90DF9174
:10231000CF911F9108950895FF920F931F93CF932C
:10232000DF938C01F62ED72FC42F222349F081E0B2
:10233000809304020E94BF199093030280930202CB
:10234000809104028823C1F08091020290910302DF
:102350000E94D719059780F0EF2DFD2FD8014C2F43
:1023600050E0CD01801B910B841795071CF48D91D3
:102370008193F7CF10920402DF91CF911F910F91BB
:10238000FF9008950E94A41B0E94EC0D0C94B01BBA
:102390000E94B41B0E947E0E0C94CE1B0E945D19FD
:1023A0000E948B1B0E94DA0D0E94C2110E94C8116C
:1023B0000E94E40DFBCFEF92FF920F931F93CF93F8
:1023C000DF938B01682F11110AC0442329F0E82FF5
:1023D000F0E0EC51FF4F6491762F862F75C0212FCE
:1023E00030E0E82FF0E0442321F0EC51FF4FE4917E
:1023F000F0E046E0049FC0011124CFEFD0E0BE0121
:102400000E94DE204BEA4603C001479F900D112435
:10241000800F911D800F911D982F990F890FAE018C
:10242000421B530B4E9FD0014F9FB00D5E9FB00DCE
:1024300011249B2F189FA0011124452F55278E0191
:10244000041B150B0E9FA0010F9F500D1E9F500DDA
:1024500011247E01E81AF108E29E8001E39E100D2E
:10246000F29E100D1124212F3327C21BD30BCE9FB8
:102470009001CF9F300DDE9F300D11246230710529
:10248000A9F048F46115710569F061307105C9F46E
:102490008B2F752F0DC06430710581F058F06630B8
:1024A000710579F47E2F8B2F932F0DC0832F7B2FF7
:1024B0009E2F09C08E2F7B2F952F05C08E2F732F37
:1024C00002C07E2F852F692FDF91CF911F910F9131
:1024D000FF90EF90089541E00E94DB1108950E9463
:1024E0006B120895CF93DF93762FE901682F842F25
:1024F0000E946F12798368838A83DF91CF91089558
:1025000080913202982F9695913021F081708260EF
:1025100080933202089588E090E00C942121CF92BC
:10252000DF92EF92FF926B017C010E948012B70153
:10253000A60188E090E0FF90EF90DF90CF900C94A0
:102540003F21E2E3F2E083E0808311828FEF828318
:102550008383148260817181828193810C948F12B4
:1025600090913602933018F49F5F9093360288233F
:1025700051F0609132027091330280913402909157
:1025800035020C948F12089581E00C94B012909152
:102590003602992319F0915090933602882351F016
:1025A0006091320270913302809134029091350231
:1025B0000C948F12089581E00C94C71270E00C9473
:1025C000FC14609105018091320280FF0AC0809165
:1025D000040123E0829FC0011124895C9D4F0C946B
:1025E000DE128091060190910701891780F7E82F8C
:1025F000F0E09F01220F331FE20FF31FE95CFD4F54
:102600001182108212828F5FF0CFE2E3F2E08081CC
:102610008E7F808360817181828193810E948F127D
:102620002FEF80E792E0215080409040E1F700C01A
:1026300000000C94E112E2E3F2E080818E7F80835F
:102640002FEF80E792E0215080409040E1F700C0FA
:1026500000000C94E1128091060281110AC081E011
:1026600080930602809132028170809305020C945F
:102670001B1308959091320290FF16C090910601AD
:1026800020910701921770F4E92FF0E0DF01AA0F03
:10269000BB1FEA0FFB1FE95CFD4F81836083428310
:1026A0009F5FF0CF0C94E1120895EF92FF920F9389
:1026B0001F93CF93DF9300D01F92CDB7DEB79091D9
:1026C000320290FF2CC0E22E142F062FF82EE92F95
:1026D000E695F0E0E358FE4F8081809308029E7FEC
:1026E000923059F49E012F5F3F4F8F2D0E9472123E
:1026F0004B8169818A810E943A13F09233020093E0
:10270000340210933502EE2051F060913202709144
:10271000330280913402909135020E948F120F9003
:102720000F900F90DF91CF911F910F91FF90EF903D
:102730000895E2E3F2E09181282F4381628188E0ED
:10274000890F0C94551380E00C94991381E00C943C
:102750009913E2E3F2E09181282F4381628188EFAF
:10276000890F0C94551380E00C94A91381E00C940C
:10277000A913E2E3F2E0628128E0620F08F46FEF50
:10278000282F438181810C94551381E00C94B91357
:10279000E2E3F2E0628128E0621B08F460E0282FA7
:1027A000438181810C94551381E00C94C813E2E3BA
:1027B000F2E0438128E0420F08F44FEF282F6281B6
:1027C00081810C94551381E00C94D713E2E3F2E07D
:1027D000438128E0421B08F440E0282F6281818178
:1027E0000C94551381E00C94E61320E00C945513DF
:1027F0008091320280FF18C0817082608093320223
:10280000662351F06091320270913302809134025C
:10281000909135020E948F124091350260913402EE
:10282000809133020C94F5130895682F81E00C9485
:10283000F81381E00C941514682F9091320296954C
:102840008FEF890F09F481E00C94F81381E00C9468
:102850001C1461E00C94F813E2E3F2E080818160E3
:10286000808386950C9429148091320280FD0C940B
:1028700005130C942C1460E00C94F813809107025B
:1028800081112CC00E94ED0C811104C00E94950D95
:102890000E94A1120E948B12609332027093330245
:1028A00080933402909335026E7F61F40E94A112EE
:1028B0000E948B1260933202709333028093340231
:1028C000909335020E9480128091320280FF03C0F3
:1028D00086950E943B1481E0809307020895E2E30D
:1028E000F2E080818160808386950C943B14109285
:1028F00006028091050281110C946F1408958823BB
:1029000011F0FA0101C0FB0109941F93CF93DF93EB
:10291000FB01128111116BC0EC010E940A0C827242
:10292000CA3CFCE5DF0709F450C0C0F4C63CECE546
:10293000DE07E1F148F4C43C9CE5D90759F178F58C
:10294000C33CDC4521F121C0C83C9CE5D90799F185
:10295000B8F546EA53E166EB73E125C0CE3CFCE5F1
:10296000DF0709F441C050F4CC3CECE5DE0791F1FF
:10297000B0F543EE53E162EF73E115C0C73D8CE55E
:10298000D807A8F1CE35DD4591F111E030C00E94A5
:1029900034142DC046E254E169E174E104C049E118
:1029A00054E166E274E10E947F1421C046EB53E1DA
:1029B00066EA73E1F8CF44ED53E165EC73E1F3CFE0
:1029C00045EC53E164ED73E1EECF42EF53E163EE8A
:1029D00073E1E9CF4BED52E164EC72E1E4CF44ECFA
:1029E00052E16BED72E1DFCF81E00E942914812F6B
:1029F000DF91CF911F9108956E9A2EB12F7B3EB13A
:102A000030644FB7F894FC01CB01880F991F680F11
:102A1000791F6E0F7F1FE617F70789F0819198E005
:102A20003EB9000000C087FF2EB9880F000000C02B
:102A300000C000C02EB900C09A9591F7ECCF4FBFEF
:102A40008FE594E00197F1F700C000000895CF935F
:102A5000DF93EC01FB018281882309F43CC1C4307F
:102A6000FDE5DF0760F4CB3F9CE5D90788F49E01C4
:102A700022503C452431310508F02EC109C0C23630
:102A8000EDE5DE0729F0C63AFDE5DF0709F024C1D0
:102A90000E94000D90932D0280932C02C1318CE591
:102AA000D80709F4C6C008F042C0C930ECE5DE071B
:102AB00009F49BC000F5C5308CE5D80709F485C042
:102AC00078F4C330ECE5DE0709F478C008F07AC08A
:102AD000C230DC4509F0F5C080912C028160EFC066
:102AE000C7309CE5D90709F478C008F07AC0809116
:102AF0002C028061E4C0CD30FCE5DF0709F487C01B
:102B000058F4CB309CE5D90709F479C008F07BC0B4
:102B100080912C0288606FC0CF30FCE5DF0709F49C
:102B200080C008F082C080912C02877FC8C0CE3F51
:102B30009CE5D90709F471C000F5C531FCE5DF0754
:102B400009F485C068F4C3319CE5D90709F475C060
:102B500008F095C00E94B70680912C028F77AFC015
:102B6000CC3FFCE5DF07A9F108F054C0CB3FDC45C2
:102B700009F0A7C080912D0240C0C230EDE5DE070C
:102B800009F489C058F4C1158DE5D80709F45AC075
:102B900008F069C080912D0282602FC0C236EDE539
:102BA000DE0709F47CC0C63AFDE5DF0709F481C001
:102BB000C330DD4509F085C080E06EC080912C02F5
:102BC00082607DC080912C0216C080912C028860AA
:102BD00076C080912D0282604FC080912C0280626D
:102BE0006EC080912C0280646AC00E94B7068091FA
:102BF0002C02806864C0846062C081603DC08091A6
:102C00002C028E7F5CC080912C028D7F58C08091F9
:102C10002C0216C080912D0218C080912D028D7F4C
:102C20002BC080912C028F7E4AC080912C028F7D18
:102C300046C080912C028F7B42C080912C02877FFE
:102C40008B7F3DC080912D028D7F8E7F15C080913E
:102C50002C0282FB222720F991E0922790FB82F937
:102C600090FB83F92CC080912D02982F9095917044
:102C70008E7F892B90FB81F980932D0222C00E94C8
:102C8000B70680912C0287FB222720F991E092273A
:102C900090FB87F914C081E00E94970D12C08091CB
:102CA0002C0284FB222720F991E0922790FB84F9E3
:102CB00006C080912C02982F909590FB80F980930C
:102CC0002C0280912C0290912D020E94110D0E94E5
:102CD000B70680E001C081E0DF91CF9108958FE8D1
:102CE00091E00197F1F700C0000008950C94A7014E
:102CF000EF92FF920F931F93CF93DF93C2E9D1E03E
:102D00000FE811E09801DE0141E050E081E0A539D3
:102D1000B80769F18D91E82FE295EF70F0E061A1BD
:102D20008F707A0102C0EE0CFF1C8A95E2F7C70192
:102D30009E2D9095962391A392A1892B82A3F901B0
:102D400081919F01E82FE295EF70F0E061A18F7013
:102D50007A0102C0EE0CFF1C8A95E2F7C7019E2D96
:102D60009095962391A392A1892B82A3CFCF0E9405
:102D70006F16E0E1F2E0B2E0E331FB0739F12991AF
:102D8000A22FA295AF70B0E090968C9190E02F703A
:102D900002C0959587952A95E2F78170D8019D919B
:102DA0008D01A92FA295AF70B0E090962C9130E0E4
:102DB0009F7002C0359527959A95E2F720FD02C0D5
:102DC00090E001C092E0892B8193D5CFDF91CF9124
:102DD0001F910F91FF90EF9008952F923F924F9285
:102DE0005F926F927F928F929F92AF92BF92CF929B
:102DF000DF92EF92FF920F931F93CF93DF9380E1C7
:102E0000682E82E0782E92E9E92E91E0F92E0FE803
:102E100011E02DE0822E22E0922ECAE0D2E0630182
:102E20005301312C212C32E0432E512CD501ED9150
:102E30005D014E2F440F440FF60141936F01D701FE
:102E40002D917D01E22FE295EF70F0E080A190E0FE
:102E50002F7002C0959587952A95E2F78170992782
:102E6000F80151918F01E52FE295EF70F0E020A17C
:102E700030E05F7002C0359527955A95E2F7F90169
:102E8000E170FF2720FF02C0E2E0F0E0E82BF92B21
:102E9000E42BD301ED933D01EF70F0E0E158FE4FDC
:102EA0009081F4018081890F808382304CF0888189
:102EB0008F5F888360E0832D0E94761621E001C039
:102EC00020E0D4018C918F3F44F488818150888325
:102ED00061E0832D0E94761621E0F4018081082EA6
:102EE000000C990BB2010E94F220D4018D934D0188
:102EF000222A33942196B3E03B1298CF822DDF91A2
:102F0000CF911F910F91FF90EF90DF90CF90BF90E6
:102F1000AF909F908F907F906F905F904F903F9079
:102F20002F900895CF93DF9386319C4541F5EB01B7
:102F30000E940A0C982F8A8120910201309103018E
:102F4000882379F09A7A81E009F480E08093130273
:102F5000911102C069E201C065E3C9010E9417191D
:102F60000AC080911302811102C069E201C065E3C9
:102F7000C9010E9419190E944C0C80E001C081E037
:102F8000DF91CF9108950F931F93CF93DF93C42FB9
:102F9000D22FFC0182818823C9F0409316020E943F
:102FA000BF19909315028093140280E28C0F883031
:102FB00008F057C0C77081E001C0880FCA95EAF7D2
:102FC000DF91CF911F910F910C94230480911602F1
:102FD000481330C080911402909115020E94D719B5
:102FE000883C910538F510E21D0FCD17B9F080E24D
:102FF0008C0F883040F4C77081E001C0880FCA95FB
:10300000EAF70E942A04183028F581E09D2F977076
:1030100001C0880F9A95EAF70E942304802F0E942E
:103020001A041830F0F4D77081E001C0880FDA95E7
:10303000EAF70AC080E28C0F883098F4C77081E00C
:1030400001C0880FCA95EAF7DF91CF911F910F91C8
:103050000C942A04802FDF91CF911F910F910C9433
:103060001A04DF91CF911F910F9108950F939C0146
:10307000CB01243F4CE5340731F188F4293DFCE5D0
:103080003F07D9F02A3D4CE5340779F1283D3C450E
:10309000A9F506E221EE41EE68ED7CE52BC0263F66
:1030A000FCE53F07E1F0A8F0273F3C4539F507E292
:1030B00025EE46EE67EF7CE51DC007E225EE45EE06
:1030C00069ED7CE517C006E221EE40EE64EF7CE599
:1030D00011C007E225EE44EE65EF7CE50BC006E289
:1030E00021EE42EE66EF7CE505C008E221E045EE08
:1030F0006AED7CE50E94C31780E008C0FC01828174
:10310000882319F01092160201C081E00F910895F2
:103110009093970180939601089590931C02809359
:103120001B020895E0911B02F0911C02309721F0E0
:103130000190F081E02D099480E00895E0911B0258
:10314000F0911C02309721F00280F381E02D099468
:1031500008952091190230911A022817390771F049
:1031600090931A0280931902E0911B02F0911C02C5
:10317000309721F00680F781E02D09940895209181
:103180001702309118022817390771F0909318022E
:1031900080931702E0911B02F0911C02309721F0FE
:1031A0000084F185E02D09940895FC01329697E0A2
:1031B00080E0915029F021912223D9F38F5FF9CF3C
:1031C0000895662349F0FC01329608962191621712
:1031D00029F0E817F907D1F780E0089581E0089514
:1031E0009C01FC0132969FEF80E04191461789F0E7
:1031F0009F3F19F4411101C0982F8F5F8630A9F7C6
:103200009F3F39F0F901E90FF11D97FDFA956283AF
:10321000089508959C012A5F3F4FFC0142814613A7
:1032200001C01282019682179307B9F708950C9492
:10323000F0180C940A19029626E0FC0111922A95C6
:10324000E9F7089508950C94221983E080931D02F4
:103250000C942319811102C081E001C082E08093A7
:103260001D020C9423190C942A1981E080931D02ED
:103270000C9423190C94351908950C943C190C9452
:103280003D190C943C190C943C190C943C190E9467
:1032900043190E9453110E94411980E00E94A2101C
:1032A000811108C081E00E94A21091E0811103C049
:1032B00090E001C091E0892F089508951F920F9228
:1032C0000FB60F9211248F939F93AF93BF9380916A
:1032D0001E02811113C08091400290914102A09181
:1032E0004202B09143024196A11DB11D809340025C
:1032F00090934102A0934202B0934302BF91AF91D9
:103300009F918F910F900FBE0F901F9018958091F5
:103310004802843031F10E94830210921E0220E4A0
:1033200088E190E00FB6F894A895809360000FBEF6
:103330002093600083B7817F846083BF83B78160FF
:1033400083BF7894889583B78E7F83BF0FB6F89438
:10335000A895809160008861809360001092600061
:103360000FBE08950E94B7060C94890282E084BDC6
:1033700093E095BD9AEF97BD80936E0008952FB7A7
:10338000F8948091400290914102A0914202B09144
:1033900043022FBF08952FB7F894609140027091B7
:1033A000410280914202909143022FBF08959C01F7
:1033B0004FB7F8948091400290914102A09142024F
:1033C000B09143024FBF821B930B089578941F92D4
:1033D0000F920FB60F9211248F939F93AF93BF93C9
:1033E0008091400290914102A0914202B09143022B
:1033F0000196A11DB11D8093400290934102A093BC
:103400004202B0934302BF91AF919F918F910F9071
:103410000FBE0F901F90189581E08093E00080E22E
:103420008093D8001092C9008FE19EE40197F1F7D4
:1034300000C0000087E090EBDC0180935102909384
:103440005202A0935302B09354029CE088E10FB65D
:10345000F894A895809360000FBE90936000FFCF12
:1034600080912A0208950895CF93DF9321E020935D
:10347000E9002FEF3091E800215035FD06C035ED11
:103480003A95F1F700002111F5CF2091E80025FFD2
:1034900014C0EC0140E050E068E070E00E94401C85
:1034A0008091E8008E778093E80088E0FE01A2E238
:1034B000B2E001900D928A95E1F7DF91CF910895E6
:1034C00080931F0270932102609320028091480232
:1034D000843001F582E08093E9008FEF9091E8005D
:1034E000815095FD06C095ED9A95F1F70000811188
:1034F000F5CF8091E80085FF0DC040E050E063E02B
:1035000070E08FE192E00E94401C8091E8008E778D
:103510008093E8000895BC0184E00C94601ABC011B
:1035200083E00C94601A089580914702811109C0CC
:103530000E94D11D0E942E1E8091E2008460809323
:10354000E20008951092470208950C943A19609190
:10355000440281E0611101C080E00C942519909132
:10356000480281E0943009F080E0609144020C94BC
:103570002A1942E061EC81E00E944A1D42E261ECBE
:1035800082E00E944A1D9091480281E0943009F047
:1035900080E0609144020C94331980914A02833098
:1035A00009F461C030F4813071F0823009F49AC0BE
:1035B00008958A3009F486C08B3009F46CC08930D4
:1035C00009F0A8C020C080914902813A09F0A2C048
:1035D0008091E800877F8093E80080914D02909170
:1035E0004E02892B21F468E082E292E003C060E0A1
:1035F00080E090E070E00E948B1C8091E8008B7767
:103600008093E800089580914902813209F082C0D8
:1036100080914D0290914E02029708F07BC08091FC
:10362000E800877F8093E8008091E80082FD05C074
:10363000809148028111F8CF6DC02091F3008091F4
:10364000F20090E0922B029731F48091F1008130EA
:1036500011F0863021F48091F10080932A0280914C
:10366000E8008B7753C080914902813A09F052C03B
:1036700080914D0290914E02892B09F04BC08091B0
:10368000E800877F8093E8008091E80080FFFCCF0E
:103690008091150136C0809149028132D9F580911F
:1036A0004D0290914E02892BA9F58091E800877F09
:1036B0008093E8000E947F1D80914B02809315014A
:1036C0000C94B70680914902813221F58091E8007F
:1036D000877F8093E8000E947F1D80914C02809339
:1036E0002B02089580914902813AA1F48091E8006B
:1036F000877F8093E8008091E80080FFFCCF809175
:103700002B028093F1008091E8008E778093E8008F
:103710000C947F1D089584B7877F84BF0FB6F894FB
:10372000A89580916000886180936000109260008D
:103730000FBE90E080E80FB6F894809361009093FC
:1037400061000FBE0C9435190E94D11D0E942E1EDF
:10375000E2EEF0E080818460808378940C94C32052
:1037600089E091E00C948D18809148028530A9F48D
:1037700080914802853079F40E9487198091460231
:103780008823B1F30E944719882391F30E942A1CD1
:103790000E94B706EDCF0C94B219089508950C94C9
:1037A000D11B292F332723303105C9F060F4213094
:1037B000310581F02230310509F044C08BE390E0FF
:1037C0002AE132E043C021323105E1F022323105F5
:1037D00049F138C082E190E025E532E037C0992711
:1037E0008130910549F028F0029761F5E4EEF1E0AF
:1037F00005C0E6E1F2E002C0EEEFF1E0849190E076
:103800009F0124C06115710541F061307105D1F44B
:1038100089E090E025E432E019C089E090E02CE2F4
:1038200032E014C06115710541F06130710551F449
:1038300082E390E027E632E009C080E490E029E9E5
:1038400032E004C080E090E020E030E0FA01318313
:103850002083089580E189BD82E189BD09B400FE1D
:10386000FDCF8091D8008F7D8093D8008091E000BB
:1038700082608093E0008091E00081FDFCCF08959C
:10388000CF92DF92EF92FF920F931F93CF93DF932C
:10389000EC018B017A010E949E1D811133C0E1145D
:1038A000F10439F0F70180819181081B190BC80FD1
:1038B000D91FC12CD12C0115110519F18091E800F7
:1038C00085FD16C08091E8008E778093E800E114B2
:1038D000F10449F0F70180819181C80ED91ED1828F
:1038E000C08285E00FC00E949E1D882321F30AC07C
:1038F00089918093F10001501109FFEFCF1ADF0A7F
:10390000DACF80E0DF91CF911F910F91FF90EF9080
:10391000DF90CF90089520914F02309150022617EA
:10392000370748F06115710539F42091E8002E77CA
:103930002093E80001C0B901FC0120E06115710588
:1039400079F1809148028823F1F18530F1F180917D
:10395000E80083FD3CC08091E80082FD2EC080918C
:10396000E80080FFEBCF2091F3008091F20090E01F
:10397000922B6115710551F08830910538F4219131
:103980002093F100615071090196F3CF21E008976F
:1039900009F020E08091E8008E778093E800CECF98
:1039A0002111CFCF0AC080914802882361F0853071
:1039B00061F08091E80083FD0AC08091E80082FFF9
:1039C000F2CF80E0089582E0089583E0089581E0D9
:1039D000089520914F02309150022617370748F082
:1039E0006115710539F42091E8002E772093E800E5
:1039F00001C0B901FC0120E06115710591F18091D0
:103A00004802882309F440C0853009F43FC0809102
:103A1000E80083FD3DC08091E80082FD2FC08091C9
:103A2000E80080FFE9CF2091F3008091F20090E060
:103A3000922B6115710559F08830910540F424915D
:103A40002093F1003196615071090196F2CF21E087
:103A5000089709F020E08091E8008E778093E800D5
:103A6000CBCF2111CCCF0AC080914802882361F0CE
:103A7000853061F08091E80083FD0AC08091E80004
:103A800082FFF2CF80E0089582E0089583E00895F8
:103A900081E00895982F973068F59093E900981782
:103AA00039F07091EC002091ED005091F00003C0CE
:103AB000242F762F50E021FD02C09F5FECCF309184
:103AC000EB003E7F3093EB003091ED003D7F309373
:103AD000ED003091EB0031603093EB007093EC001F
:103AE0002093ED005093F0002091EE0027FDE5CFEC
:103AF00080E008958F708093E90081E008958091BF
:103B0000490287FF11C08091E80082FD05C08091C5
:103B100048028111F8CF11C08091E8008B770BC06B
:103B200080914802882349F08091E80080FFF8CF17
:103B30008091E8008E778093E80008952091E4005A
:103B40003091E50095E64091EC00842F817040FFB4
:103B500023C08091E80080FD1DC080914802882329
:103B600099F0853099F08091EB0085FD11C040916E
:103B7000E4005091E5002417350729F3915011F026
:103B80009A01E1CF84E0089582E0089583E00895EA
:103B900081E0089580E008954091E80042FFDDCF84
:103BA00008950E943F1E0E94471EE0EEF0E08081D3
:103BB00081608083E8EDF0E080818F77808319BC9D
:103BC000A7EDB0E08C918E7F8C9380818F7E808377
:103BD0001092470208950F931F93CF93DF930E9493
:103BE0003F1E0E94471EC8EDD0E088818F778883F2
:103BF00088818068888388818F7D888319BC109232
:103C0000480210924402109246021092450200EEC1
:103C100010E0F80180818B7F8083888181608883B8
:103C200042E060E080E00E944A1DE1EEF0E0808129
:103C30008E7F8083E2EEF0E08081816080838081EE
:103C400088608083F80180818E7F80838881806195
:103C50008883DF91CF911F910F910895E8EDF0E0F7
:103C600080818F7E8083E7EDF0E0808181608083BA
:103C700084E082BF81E0809347020C94EB1DE8ED65
:103C8000F0E080818E7F80831092E2000895109290
:103C9000DA001092E10008951F920F920FB60F9272
:103CA00011242F933F934F935F936F937F938F9341
:103CB0009F93AF93BF93EF93FF938091E10082FFB7
:103CC0000BC08091E20082FF07C08091E1008B7FF2
:103CD0008093E1000E94C2208091DA0080FF1FC023
:103CE0008091D80080FF1BC08091DA008E7F809386
:103CF000DA008091D90080FF0DC080E189BD82E1AA
:103D000089BD09B400FEFDCF81E0809348020E9486
:103D1000941A05C019BC109248020E94A21A809100
:103D2000E10080FF19C08091E20080FF15C0809102
:103D3000E2008E7F8093E2008091E20080618093B8
:103D4000E2008091D80080628093D80019BC85E0A1
:103D5000809348020E94A71A8091E10084FF30C03E
:103D60008091E20084FF2CC080E189BD82E189BDA1
:103D700009B400FEFDCF8091D8008F7D8093D800DC
:103D80008091E1008F7E8093E1008091E2008F7E40
:103D90008093E2008091E20081608093E200809154
:103DA0004402882311F084E007C08091E30087FD7E
:103DB00002C081E001C083E0809348020E94AF1AF4
:103DC0008091E10083FF29C08091E20083FF25C03C
:103DD0008091E100877F8093E10082E08093480238
:103DE000109244028091E1008E7F8093E1008091E7
:103DF000E2008E7F8093E2008091E20080618093F8
:103E0000E20042E060E080E00E944A1D8091F00004
:103E100088608093F0000E94A51AFF91EF91BF91F6
:103E2000AF919F918F917F916F915F914F913F9152
:103E30002F910F900FBE0F901F9018951F920F9209
:103E40000FB60F9211242F933F934F935F936F936D
:103E50007F938F939F93AF93BF93CF93DF93EF9312
:103E6000FF93C091E900CF708091EC00D82FD17002
:103E700080FDD0E81092E9008091F000877F809368
:103E8000F00078940E94621F1092E9008091F00087
:103E900088608093F000CD2BCF70C093E900FF9134
:103EA000EF91DF91CF91BF91AF919F918F917F91D2
:103EB0006F915F914F913F912F910F900FBE0F9097
:103EC0001F9018951F93CF93DF93CDB7DEB7AA97B6
:103ED0000FB6F894DEBF0FBECDBFE9E4F2E08091EB
:103EE000F100819322E0E135F207C9F70E94CD1A73
:103EF0008091E80083FF2EC18091490290914A028F
:103F0000492F50E04A30510508F024C1FA01EE591A
:103F1000FF4F0C940621803821F0823809F01AC135
:103F200008C08091450290914602992389F08260F1
:103F30000FC080914D028F70873008F00BC18093C5
:103F4000E9008091EB0085FB882780F91092E90059
:103F50009091E800977F9093E8008093F100109291
:103F6000F100D1C0282F2D7F09F0F4C0882319F06B
:103F7000823061F0EFC080914B02813009F0EAC0DD
:103F8000933009F080E0809346022EC080914B026E
:103F900081112AC080914D028F702FEF280F26309B
:103FA00008F0D8C08093E9002091EB0020FF1CC0EE
:103FB000933021F48091EB00806214C09091EB006B
:103FC00090619093EB0021E030E0A90102C0440F22
:103FD000551F8A95E2F74093EA001092EA0080911B
:103FE000EB0088608093EB001092E9008091E8007C
:103FF000877F8093E8000E947F1DACC08111AAC01A
:1040000010914B021F778091E3008078812B809381
:10401000E3008091E800877F8093E8000E947F1D85
:104020008091E80080FFFCCF8091E300806880935E
:10403000E300111102C082E001C083E080934802D6
:1040400089C08058823008F085C080914B029091E1
:104050004C028C3D53E0950779F583E08A838AE230
:1040600089834FB7F894DE01139620E03EE051E2D9
:10407000E32FF0E050935700E49120FF03C0E29556
:10408000EF703F5FEF708E2F90E0EA3010F0C79630
:1040900001C0C0968D939D932F5F243149F74FBF88
:1040A0008091E800877F8093E8006AE270E0CE01AB
:1040B00001960E948B1C16C060914D0270914E02B9
:1040C000AE014F5F5F4F0E94CF1BBC01892B09F4EB
:1040D00041C09091E800977F9093E80089819A8190
:1040E0000E94E91C8091E8008B778093E80032C041
:1040F000803881F58091E800877F8093E800809187
:1041000044028093F1008091E8008E7772CF811194
:1041100021C080914B0290914C0299270297D4F4D0
:104120008091E800877F8093E80080914B02809324
:1041300044020E947F1D80914402811106C080913B
:10414000E30087FD02C081E001C084E08093480263
:104150000E94B91A8091E80083FF0AC08091E800AC
:10416000877F8093E8008091EB0080628093EB0072
:10417000AA960FB6F894DEBF0FBECDBFDF91CF91E8
:104180001F9108950895CF93809148028823A1F04C
:10419000C091E900CF709091EC00892F817090FD63
:1041A00080E8C82B1092E9008091E80083FD0E940E
:1041B000621FCF70C093E900CF910895AA1BBB1B6B
:1041C00051E107C0AA1FBB1FA617B70710F0A61B17
:1041D000B70B881F991F5A95A9F780959095BC0138
:1041E000CD01089597FB072E16F4009407D077FDB4
:1041F00009D00E94DE2007FC05D03EF49095819501
:104200009F4F0895709561957F4F0895EE0FFF1FA2
:104210000590F491E02D0994FB01DC0104C08D911F
:104220000190801921F441505040C8F7881B990B28
:104230000895F999FECF92BD81BDF89A992780B56E
:104240000895A6E1B0E044E050E00C945321A8E1C9
:10425000B0E042E050E00C945321262FF999FECFB4
:1042600092BD81BDF89A019700B4021639F01FBAC9
:1042700020BD0FB6F894FA9AF99A0FBE08950396E6
:10428000272F0E942E210E942D21252F0E942E21B2
:10429000242F0C942E210196272F0E942E210C945E
:1042A0002D21DC01CB01FC01F999FECF06C0F2BD46
:1042B000E1BDF89A319600B40D9241505040B8F7E4
:0642C0000895F894FFCF01
:1042C600C800E9010003000303301A341A931A8F59
:1042D6001A8B1A331A01E200E900EA00B500B600AB
:1042E600B700CD008301CC008A019201940121021E
:1042F600230224022502260227022A02B300B40062
:104306006F007000818283E200E900EA00B500B622
:1043160000B700CD008301CC008A019201940121EF
:1043260002230224022502260227022A02B300B42F
:10433600006F007000818283F036359367000100BC
:10434600FF0100010000FFFF0000010001FF003136
:06435600373432339500FC
:00000001FF
